:020000040000FA
:020000001628C0
:040002000034003492
:08000800F0000308F1000B19E0
:100010000123831203130C180D23831203138C186E
:0C002000062371088300F00E700E09002A
:04002C008316031321
:100030000510851005118515051685160513851300
:1000400006148614061186110612861206138613EC
:1000500086308100E0308B0003308C00EF3092005E
:100060008312031307309F00013090000730920085
:1000700085018601A001A801BD011630D422230804
:10008000BC001930D4222308C5001730D42223081D
:10009000C0001830D4222308C1001030D422230815
:1000A000C2001130D4222308C300692197221430E2
:1000B000D4222308A9001530D4222308AA00123024
:1000C000D4222308A6001330D4222308A700B52089
:1000D0003722A5010030A40064002508D42224089A
:1000E000B7222308C522A50AA40A2408083A031D3A
:1000F0007B284030A4002408483A031D6C282013B4
:100100003030A4006400201F82282013A40B822812
:10011000A010BD01AE21A0136400461A9B2806184A
:100120009528461546169101121586189B28C61566
:100130004616910112158B132008C400851AC416A7
:10014000851EC4122008C406031D69218B17831263
:100150000313051A2011A01DB028A011B520AE214F
:10016000A01C8C28A0101A218C28451CE5283E1FB5
:10017000CC2883120313201246302702BA00031C36
:100180000B30031C201603180A302602BB00201E69
:10019000CB289C30BA02EB282608BB002808B900FF
:1001A0002708BA000530B9073908633C0318DB2873
:1001B000BA0A6430B9022D30BA073A08633C031812
:1001C000E428BB0A6430BA02EB282608BB002808E2
:1001D000B9002708BA00BE1E0A29B701B80150307D
:1001E000A4003B08B8070318B70AA40BF128643031
:1001F000A400AB01AC013A08AB070318AC0AA40B8E
:10020000FB287D30AD00AE01DD222B08B8070318B6
:10021000B70A1829B701B8016430A4003B08B80731
:100220000318B70AA40B0E293A08B8070318B70A2F
:100230007C210800640083120313851923292908EF
:10024000A600A7012015461D452946112011A0151D
:10025000BE1A2C29A80133291930A8020318332902
:100260004B30A800A703A7032708633C03184529C0
:100270006330A700A6032608290203194529031C99
:1002800045292A08A6006330A70020194929C61D60
:100290006829C6192011C611A015BE1A5129A80136
:1002A00059291930A8072808633C03185929A801BF
:1002B000A70AA70A2708633C03186829A701A60A0A
:1002C00026082A02031868292908A600A701A80100
:1002D000080083120313851A7429A0124008B7007E
:1002E000BE004108B8007A29A0164208B700BE0037
:1002F0004308B8007C2108008514A9210514A92110
:100300000510A9210830B600B71B0515B71F051148
:10031000A9210514A9210510A921B70DB60B84291F
:100320000830B600B81B0515B81F0511A921051422
:10033000A9210510A921B80DB60B92290511A921F3
:100340008510A921A9210514A9210510A921A921F8
:1003500008000A30B500B50BAB2908003E1BB529D3
:100360000030B7224130C522B9290030B7224630CB
:10037000C5220130B7224D30C5220230B7222030CD
:10038000C5222608AB00AC016430AD00AE01DD2211
:100390000330B7222B080026C5222D08AB000A30F7
:1003A000AD00AC01AE01DD220430B7222B080026DF
:1003B000C5220530B7222D080026C5223E1FE5299B
:1003C0000630B7222C30C522E9294030B7222C3024
:1003D000C5222708AB00AC010A30AD00AE01DD221A
:1003E0003E1FF8290730B7222B080026C522FD2919
:1003F0000630B7222B080026C5223E1F052A4030B2
:10040000B7222D080026C5220A2A0730B7222D0858
:100410000026C5222808AB00AC010A30AD00AE01B1
:10042000DD224130B7222B080026C5224230B722F8
:100430002D080026C5224330B7222030C5223E1F9A
:10044000262A4430B7224D30C5222A2A4430B7220A
:100450006B30C5224530B7224830C5224630B7221E
:100460007A30C5224730B7222030C52208008312D7
:1004700003138611810120106400201C3C2A2010E7
:10048000810120106400201C422A20100611000067
:1004900086153C30A2009C22201081016400861148
:1004A0006400201C502A640086152010E030810072
:1004B00064008611201C5A2A6400861520106400EE
:1004C0000000861197229722640006113C30A2009A
:1004D00086159C22640000008611972297226400F2
:1004E000061186150C30A2009C22640000008611C3
:1004F0009722972264002010061186150130A20071
:100500009C226400000086112010AA308100201C6B
:10051000872A64002010061186150630A2009C224E
:1005200064000000861197229722640008001030B2
:10053000A100A10B992A08008312031305110510CD
:100540008513051386130613861206122218051545
:10055000A218051422198517A2190517221A861741
:10056000A21A0617221B8616A21B06160800A20056
:10057000A217D2228611D2220611D2228615D222A9
:100580009C22D222861197220800A200D222861134
:10059000D2220615D2228615D2229C22D222861180
:1005A0009722080000000800831603139B001C1408
:1005B0001A0883120313A30008001030B100AF0122
:1005C000B001AB0DAC0DAF0DB00D2F08B20030086F
:1005D000B3002D08AF02031C2E0A03182E08B00228
:1005E0000318F62A3208AF003308B000031C2B10A2
:1005F00003182B14B10BE12A2F08AD003008AE0010
:1006000008000B1183120313201408008C108312AE
:100610000313A0171211461208000C1020173C30CB
:100620008F00BD0A3D083C06031D1A2B83120313DD
:10063000A014BD013C08031D1F2BA014BD01080020
:100C0000013EB4000030B40707300318013E8A00EB
:060C100034080027080073
:100E0000820030343134323433343434353436348F
:060E100037343834393498
:02400E00543F1D
:1042000023002A002000410068006F006A0020009F
:104210005A004100570049004E0020002A002300A8
:10422000FD004500910039008C0096000300BD00A0
:044230004500010044
:00000001FF
